:020000040800F2
:10000000C806002091010008610A00085D0A000886
:100010005F0A000831070008F11300080000000023
:10002000000000000000000000000000E10D0008DA
:10003000AD08000800000000FD0A00086D0E000871
:10004000AB010008AB010008AB010008AB010008E0
:10005000AB010008AB010008B1080008AB010008C3
:10006000AB010008AB010008AB010008AB010008C0
:10007000AB010008AB010008AB010008AB010008B0
:10008000AB010008AB010008AB010008AB010008A0
:10009000AB010008AB010008AB010008AB01000890
:1000A000AB010008AB010008AB010008AB01000880
:1000B000AB010008AB010008AB010008AB01000870
:1000C000AB010008AB010008AB010008AB01000860
:1000D000AB0100083D120008AB010008AB010008AD
:1000E000AB010008AB010008AB01000800F002F80A
:1000F00000F03EF80AA090E8000C82448344AAF184
:100100000107DA4501D100F033F8AFF2090EBAE881
:100110000F0013F0010F18BFFB1A43F0010318473B
:100120001C1A00003C1A0000103A24BF78C878C19D
:10013000FAD8520724BF30C830C144BF04680C60ED
:10014000704700000023002400250026103A28BF35
:1001500078C1FBD8520728BF30C148BF0B60704739
:100160001FB59DE8030000F0BFF81FBD10B510BD1E
:1001700000F03CF91146FFF7F3FF01F060FC00F0DE
:100180007BF903B4FFF7F2FF03BC01F055FC00005C
:100190000948804709480047FEE7FEE7FEE7FEE71B
:1001A000FEE7FEE7FEE7FEE7FEE7FEE70448054957
:1001B000054A064B70470000850E0008ED00000858
:1001C000C8000020C8060020C8020020C802002085
:1001D0007047002000F061F8FFF7C8FF012001F030
:1001E0002BFC10B5203AC0F00B80B1E81850203A33
:1001F000A0E81850B1E81850A0E81850BFF4F5AFC7
:100200005FEA027C24BFB1E81850A0E8185044BF50
:1002100018C918C0BDE810405FEA827C24BF51F8BD
:10022000043B40F8043B08BF7047D20728BF31F8B1
:10023000023B48BF11F8012B28BF20F8023B48BF02
:1002400000F8012B704770477047704770B504463F
:10025000051F00F029F80068002C14BF446870BD29
:10026000002C18BFAC423CBF20466468F8D301683C
:100270000A18AA4218BF456003D12A6805461144EE
:10028000016028684119A1421CBF6C6070BD6168A3
:10029000696021680844286070BD10B500F088F8D6
:1002A000BDE8104000F07EB8004870476C000020A8
:1002B00000487047980000207047704770477047AB
:1002C00038B504460A4600206946AFF3008000288E
:1002D00008BF38BD02460099204600F0B3F801205F
:1002E00038BD012000F0E7B8F8B5AFF3008005464F
:1002F00000200C46102000BF0646A819A0420DD9C8
:10030000324669460020AFF30080070008BF00F0C6
:10031000D2F80098A04218BF0546C419FFF7C4FFE1
:1003200005600746F01D20F007004619284600F03A
:1003300082F8B44208BFF8BDA21B31463868BDE858
:10034000F84000F07FB870B50646FFF7ADFF0568CE
:1003500006F10B0020F00704B4429CBF002070BDE2
:100360002B466A68BAB11068A04210D304F10801A4
:1003700088423CBF5068586007D3516810194160EB
:100380001168091B016058601460101D70BD134690
:100390005268002AE7D121462846FFF791FF00283E
:1003A000DED170BD002801D001F046BB70470000CF
:1003B00010B5002102A000F065F8012010BD00007A
:1003C000534947414252543A2041626E6F726D6107
:1003D0006C207465726D696E6174696F6E000000E7
:1003E00000F070B800487047640000207546FFF7C1
:1003F000F9FFAE4605006946534620F007008546E2
:1004000018B020B5FFF7D2FEBDE820404FF000063F
:100410004FF000074FF000084FF0000B21F00701EC
:10042000AC46ACE8C009ACE8C009ACE8C009ACE82F
:10043000C0098D46704700210160C0E90110704776
:1004400010207047034640688C46002818BF884239
:100450003CBF03464068F8D318681844884207D068
:100460000CF1030020F00700001D411A521A01464A
:10047000081D0A60FFF7EABE0446AFF3008020467D
:10048000FFF77FFE70B505460C460A2000E06D1CA4
:1004900001F0D3FA35B128780028F8D102E0641CC5
:1004A00001F0CBFA14B120780028F8D1BDE87040F3
:1004B0000A2001F0C2BA10B500F012F8BDE81040F1
:1004C000FFF770BF10B500F036F8016919B10022CE
:1004D0000261884701E080688047FFF77AFE0000EC
:1004E00010B5012805D0002103A0FFF7CBFF0120A4
:1004F00010BD09A1F8E7000053494752544D454D3E
:100500003A204F7574206F662068656170206D65B4
:100510006D6F7279000000003A2048656170206DAF
:10052000656D6F727920636F7272757074656400A7
:1005300010B5FFF74EFE70B500F022F804680546CE
:10054000A4B92020FFF7FFFE040011D009490020C4
:100550002C60C4E900010849A1602073206160613A
:100560000649A06109B100F00FF8E061204670BDB6
:10057000FFF72FFE0000000031050008000000001A
:1005800000487047A000002010B58820FFF7DBFE70
:10059000002801D00021017010BD802902D808B1C7
:1005A000017809B100207047012100F8081B70474D
:1005B00018B100F10802914201D0002070470021DB
:1005C000017070470029816802D041F0010101E00B
:1005D00021F00101816070470D4910B5884202D1B8
:1005E000012144150AE00B49884202D1012104157A
:1005F00004E0094988420AD10121CC03204600F0D9
:10060000B9FA2046BDE81040002100F0B3BA10BD91
:100610000024014000280140003C0140002981687D
:1006200002D041F4801101E021F480118160704713
:10063000014600208968490700D501207047C06C39
:1006400080B270470246002012680A4200D00120A2
:100650007047014600208968090700D501207047CE
:1006600010B542680E4B1A40D1E9003442EA042228
:100670001343436083680B4A1340D1E9034222438A
:100680008C6843EA44031A438260C26A097D22F4FB
:100690007002491EC9B242EA0151C16210BD000098
:1006A000FFFEF0FFFDF7F1FF70B5072409290AD915
:1006B000C568A1F10A0606EB4606B440A543B3405F
:1006C0001D43C56007E0056901EB4106B440A54341
:1006D000B3401D4305611F23072A09D2446B521EF4
:1006E00002EB820293409C4391400C43446370BDF3
:1006F0000D2A09D2046BD21F02EB820293409C4365
:1007000091400C43046370BDC46A0D3A02EB82024F
:1007100093409C4391400C43C46270BD816841F09A
:10072000080181607047816841F004018160704771
:10073000FEE70000044A01238340106809B1184312
:1007400000E09843106070470074004010B501212C
:100750004C07204600F0F6F92046BDE81040002185
:1007600000F0F0B930B5084C236840F6FE728240C4
:100770009343D1E900252A43D1E902510D432A438D
:1007800082401A43226030BD00740040034A08B51D
:10079000104408300090016008BD00000074004063
:1007A000034A08B5104414300090016008BD0000F1
:1007B00000740040044A0029516801D0014300E060
:1007C0008143516070470000002004E0016821F07F
:1007D000010101600021016041608160C160314917
:1007E000304A0839904203D1486840F00F0006E0D3
:1007F0002C4A1432904204D1486840F0F00048601E
:100800007047284A2832904203D1486840F470600B
:10081000F5E7244A3C32904203D1486840F47040E6
:10082000EDE7204A5032904203D1486840F47020EE
:10083000E5E71C4A6432904203D1486840F47000F6
:10084000DDE7184A7832904203D1486840F0706082
:10085000D5E7154A111F904203D1086840F00F00F8
:1008600006E0114A1432904204D1086840F0F000CA
:10087000086070470C4A2832904203D1086840F45F
:100880007060F5E7084A3C32904203D1086840F4B2
:100890007040EDE7044A50329042EAD1086840F4D3
:1008A0007020E5E70800024008040240704700009D
:1008B00002490120087000F003B800004000002049
:1008C00001490860704700001404014030B51A491E
:1008D000C368026853B30B6893430B600A1D136827
:1008E0000468A343136042680A44136804682343FE
:1008F0001360114A083213680468A3431360131D80
:100900001C680568AC431C608468102C05D0214429
:100910000A68006802430A6030BD11680468214318
:100920001160196800680143196030BD40680844CF
:1009300001689143016030BD0004014010B58A0791
:1009400021F003040649130F21440F228C689A40BA
:1009500094438C608A68984002438A6010BD00000E
:1009600000000140F0B50A7A002502F00F03D2061C
:1009700001D54A6813430C784FF00F0E0122ECB1F9
:10098000D0F800400F8802FA05F63740B74211D17F
:100990004FEA850C0EFA0CF724EA070703FA0CF469
:1009A0003C438F68282F02D0482F02D002E04661D6
:1009B00000E006616D1C082DE4D304600C88FF2C58
:1009C0001ED944685FF0000606F1080702FA07F531
:1009D0000F882F40AF420FD14FEA860C0EFA0CF76A
:1009E000BC4303FA0CF73C438F68282F00D14561C4
:1009F0008F68482F00D10561761C082EE4D344602F
:100A0000F0BD0000F0B5144C002801DAE36900E005
:100A10006368420D120185B2C0F301579540C0F3DF
:100A20000346032F05D0C2020AD50322B2409343E6
:100A300007E023F07062636823F07063636002E094
:100A4000AB4343F0706201B12A43002801DAE2614E
:100A5000F0BD6260F0BD000000000140FEE7FEE76F
:100A6000FEE70000F0B50F210278446801234FF043
:100A7000E026DCB1124C2468457804F4E064C4F547
:100A8000E064240AC4F10407E1408478BD400C40CE
:100A90002C4321010B4C1155007800F01F018B40B5
:100AA000400906EB8000C0F80031F0BD02F01F00E5
:100AB0008340500906EB8000C0F88031F0BD000093
:100AC0000CED00E000E400E00A4B1A6822F003029B
:100AD00002431A600848026842F0040202600129D9
:100AE00005D020BF016821F004010160704730BFCC
:100AF000F8E700000070004010ED00E070470000D3
:100B0000034A516821F4404101435160704700009D
:100B100000100240044A0029516901D0014300E05D
:100B2000814351617047000000100240044A0029CF
:100B3000D16901D0014300E08143D16170470000D9
:100B400000100240044A0029116901D0014300E06D
:100B5000814311617047000000100240044A0029DF
:100B6000916901D0014300E0814391617047000029
:100B700000100240044A0029D16801D0014300E07E
:100B80008143D160704700000010024030B5214918
:100B90004A6812F00C03204A03D0042B01D0082B22
:100BA00001D0026015E04B684C6803F470134FF0FD
:100BB000020514F4803F05EB934307D0CC6A04F0A0
:100BC0000F04641CB2FBF4F25A43EAE7134A53439E
:100BD00003604A680F23124C03EA1212A35C0268F6
:100BE000DA4042604B68072505EA1323E35C22FAEA
:100BF00003F383604B6805EAD323E35CDA40C26009
:100C00004968032303EA9131231F595CB2FBF1F1D8
:100C1000016130BD0010024000127A0000093D0061
:100C2000460000200246002053090949012B0BD041
:100C3000022B0BD0D1F8241002F01F0201239340A5
:100C40000B4200D0012070470968F5E7096AF3E715
:100C5000001002400248406800F00C00704700009D
:100C6000001002400B490A6822F480320A600A68C8
:100C700022F480220A60B0F5803F07D0B0F5802FC3
:100C800003D1086840F4A02008607047086840F469
:100C90008030F9E700100240014908667047000003
:100CA00000004242034A516821F0030101435160B0
:100CB000704700000010024018B500204FF4A064F7
:100CC00000903120FFF7AEFF0099491C0091A1422E
:100CD00001D00028F5D03120FFF7A4FF002800D074
:100CE000012018BD3EB504460B48012150F82400F0
:100CF000FFF734FF084869460A3830F81400ADF8A9
:100D000000001020029003200190044850F82400B5
:100D1000FFF728FE3EBD0000D81A0008040000209E
:100D20000349044A31F8101052F82000416170471D
:100D3000CE1A0008040000200349044A31F81010BC
:100D400052F8200001617047CE1A0008040000200C
:100D500030B5044620480D4689B050F824000121E2
:100D600040F00100FFF7FAFE042008901A4806A997
:100D70000C3830F81400ADF81800184850F824006A
:100D8000FFF7F0FD012D24D11348103810F814108E
:100D9000801C10F81400FFF7D1FD0F480A3830F816
:100DA00014000090002001900820CDE9020568465B
:100DB000FFF78CFD0848083810F814008DF8100073
:100DC0000F208DF811008DF8120004A80595FFF78B
:100DD00049FE09B030BD0000D41A00080000002010
:100DE000704700000CB500211F4801910091026876
:100DF00042F4803202604FF4A063026802F40032D1
:100E00000092019A521C0192009A12B9019A9A42D8
:100E1000F3D10268920324D5012100914168416019
:100E20004168416041684160416821F47C11416042
:100E3000416841F498114160016841F0807101609E
:100E400001688901FCD5416821F0030141604168D6
:100E500041F0020141604168C1F381010229FAD1E8
:100E60000CBD00910CBD0000001002400448407809
:100E700000284FF0000001D0FFF75EBFFFF750BF22
:100E800040000020104810B5016841F001010160E8
:100E900041680E4A1140416001680D4A11400160ED
:100EA000016821F480210160416821F4FE01416064
:100EB0004FF41F0181600021C162FFF793FF0549D4
:100EC0004FF00060086010BD001002400000FFF805
:100ED000FFFFF6FE08ED00E00029018802D041F096
:100EE000800101E021F08001018070470029018824
:100EF00002D041F0010101E021F0010101807047C1
:100F0000002930F8441F02D041F4004101E0C1F350
:100F10000E010180704700004B4910B5884202D194
:100F20000121C41486E0B0F1804F09D047498842BE
:100F30000DD101210220FFF705FE0021022064E00F
:100F400001210846FFF7FEFD002101205DE0404938
:100F5000884206D101210420FFF7F4FD002104207E
:100F600053E03C49884206D101210820FFF7EAFD01
:100F70000021082049E03849884206D1012110208B
:100F8000FFF7E0FD002110203FE03449884206D100
:100F900001212020FFF7D6FD0021202035E0304937
:100FA000884202D10121441444E02E49884202D1F2
:100FB0000121CC043EE02C49884202D101210C05DC
:100FC00038E02A49884202D101214C0532E0284903
:100FD000884206D101214020FFF7B4FD00214020C6
:100FE00013E02449884206D101218020FFF7AAFDA1
:100FF0000021802009E0204988420AD1841501217E
:101000002046FFF79FFD00212046BDE81040FFF776
:1010100099BD1A49884202D101210C040AE01849FD
:10102000884202D101214C0404E0164988420AD1C9
:1010300001218C042046FFF79DFD2046BDE81040AD
:101040000021FFF797BD10BD002C014000040040B7
:1010500000080040000C0040001000400014004058
:1010600000340140004C0140005001400054014058
:1010700000180040001C00400020004000400140DB
:10108000004401400048014070B5028C22F010027B
:101090000284028C8488038B0D8823F4E6464FF685
:1010A000FF7303EA052535430E8922F0200203EA87
:1010B000061616434A8803EA02123243104EB04223
:1010C00002D0104EB04215D122F080064A8924F495
:1010D000406403EA0212324322F040068A8803EA9F
:1010E000021232438E8903EA86062643CC8903EA3C
:1010F0008404344384800583C9880187028470BDD9
:10110000002C01400034014070B5028C22F4805262
:101110000284048C8288838B0D8823F4E6464FF684
:10112000FF7303EA0525354324F400560C8903EACE
:10113000043434434E8803EA06362643094CA04261
:1011400002D0094CA04205D122F480448A8903EAE6
:101150008212224382808583C988A0F840100684C9
:1011600070BD0000002C014000340140828B4FF61E
:10117000FF7322F4006203EA012111438183704767
:1011800081857047A0F840107047000030B5028894
:101190001B4B1C4C98420DD0A0420BD0B0F1804F9D
:1011A00008D0194DA84205D0184DA84202D0184DBC
:1011B000A84203D122F070054A882A43154DA8425F
:1011C00006D0154DA84203D022F44075CA882A43A0
:1011D00002808A8882850A88028598420AD0A042C5
:1011E00008D00E4A904205D00D4A904202D00D4AD6
:1011F000904201D1097A01860121818230BD00002F
:10120000002C014000340140000400400008004070
:10121000000C00400010004000140040004001405D
:1012200000440140004801404FF6FF7181800021D9
:101230000180C18041800172704700000E4810B5E6
:101240000188890616D5018821F020010180011D41
:1012500009880A4CCAB26168094B0B44491C616099
:101260001A70712A06D100216160322100F0B5F8B0
:101270000120207010BD0000003801400C0000204B
:101280005800002010B5038A4FF2FF0213400A886D
:101290004C8822438C88C9880C4322431A4302821B
:1012A00010BD0021018041808180C18070470029EC
:1012B000818902D041F4005101E021F40051818183
:1012C0007047002A828A01D00A4300E08A43828262
:1012D00070470246002012880A4200D00120704761
:1012E00010B5C1F3421301F01F040121A140012BED
:1012F00007D0022B07D01430002A026805D00A4319
:1013000004E00C30F8E71030F6E78A43026010BDC5
:1013100030B50446008A85B00D464CF6FF71084092
:10132000E98801432182A1894EF6F3100140A88883
:101330002A8910436A890A431043A081A08A4FF684
:10134000FF410840A9890143A1826846FFF71EFCBE
:101350001B48844201D1039800E00298A189090446
:10136000002900EBC00101EB0010296802DA4FEA06
:10137000410101E04FEA8101B0FBF1F06422B0FBD2
:10138000F2F14FEA01114FEA11136FF018056B43A8
:1013900000EB8300A3891D044FF0320306D503EB55
:1013A000C000B0FBF2F000F0070005E003EB001016
:1013B000B0FBF2F000F00F000843208105B030BD13
:1013C000003801404FF41651016000218180C18036
:1013D00001810C2242818181704700B50346C8B269
:1013E000988080211846FFF774FF0028F9D000BDCF
:1013F000FEE72DE9F041827D86880023012A12D183
:10140000C269941CC0E906241180B0F814C00469B4
:10141000C26904EB4C01914200D1C461002117E084
:1014200082888A4201D8FEF7D4FE056835F911702A
:101430008569AA1E8261B5F90050A24205D26FF0FB
:10144000010202EB4C022244826107FB0533491C76
:10145000B142E5D343F3CF30BDE8F08170B50B0462
:101460001B0C026083804FF0000585718260C260B2
:1014700019D000F110048EB2700000F0C5FA20609F
:101480000120A680A0712068A060E060B0B2AA1E12
:10149000216802EB40021144401E21F80259FBD1A1
:1014A000A4F1100070BDFEF794FE0446032100F085
:1014B000A1F804F582700121054600F053F904F506
:1014C000887604F58074284600F078FA01B2304638
:1014D000FFF78FFF00F5006081B2204600F07EFA32
:1014E000F1E7000010B5012100F0C4F807490160E0
:1014F00000F58870064A1F21FFF7B0FFA0F5887439
:1015000064210C3800F0EEF8204610BD241B0008C2
:10151000841A000810B50649016000F5907000F0CB
:10152000A7FA103800F0A4FAA0F5887010BD0000EA
:10153000241B000810B5064904460020087002214B
:101540000120FFF7C1FA2046BDE8104000F076B850
:101550004000002030B58BB001210220FFF7E6FAF1
:101560004FF40070ADF81C0018200990022008907C
:1015700007A91D48FFF7F6F901211C48FFF742FAB9
:101580001B4D2846FFF7C8FC42F6E060ADF814009A
:101590004FF47A70ADF810000024ADF81640ADF8A5
:1015A000124004A92846FFF7F1FD6020ADF80000C5
:1015B0000120ADF8020041F27070ADF80600ADF800
:1015C000084069462846FFF79FFD08212846FFF797
:1015D000CDFD01212846FFF77FFC01212846FFF7BA
:1015E00085FC0BB030BD000000100140000C1A005B
:1015F0000004004070B5052901DBFEF7EAFD0D4847
:1016000099B10D4A054632F811400121FFF76EFCF1
:101610004FF6FF7000EA44012846FFF7B1FD21466E
:101620002846BDE87040FFF7ADBDBDE87040002121
:10163000FFF75CBC00040040101B000810B5044616
:101640004FF48030FFF70EFBFFF736FBC4F80C01B8
:1016500001280DD1FFF720FB3920FFF7E3FA00281E
:10166000FAD00220FFF71EFBFFF7F4FA0828FBD19F
:1016700010BD000010B50C46194902C000F032F947
:1016800000222146FC3000F0EFF805222146001D23
:1016900000F06CF8A0F5827472B60020FFF722FB10
:1016A0000020FFF73DFB0120FFF71CFB0120FFF7A7
:1016B00037FB01210020FFF74BFB01210846FFF714
:1016C00079F801210220FFF775F80121C802FFF720
:1016D00071F82046FFF73EFF62B6204610BD0000BD
:1016E000341B000810B504464FF6FF7088B08142E5
:1016F00001D3FEF76EFDA1806846FFF795FDA08837
:10170000ADF804001820ADF800000020ADF8060088
:10171000ADF8020069462068FFF738FD6020ADF89B
:101720000C000120ADF80E00A088ADF812000220D8
:10173000ADF8140003A92068FFF7A6FC012120687A
:10174000FFF7DEFB08B010BD10B54FF6FF729142F7
:1017500001D3FEF73EFD4FF47A72BDE810405143CD
:10176000FFF7C0BF0068FFF7C1BB000070B50546BA
:101770008AB04FF0804028600C46AA8001214015B5
:10178000FFF7ECF90020FFF7BBF93448002CD0E953
:10179000031240690691CDE9072052D0012C52D0A6
:1017A000022C01D0042C50D05FF00400ADF81800DA
:1017B00006A92B48FFF7D6F8F4B3012C49D0022C28
:1017C00001D0042C47D00226264C2046FEF704FF09
:1017D0002249182218316846FEF703FD6946204663
:1017E000FEF73EFF0723012231462046FEF75CFF4D
:1017F00001212046FEF712FF01210846FFF796F966
:10180000A9882846FFF7A0FF01212046FEF7DAFE4F
:1018100000212868FFF76AFB2046FEF77FFF20467D
:10182000FEF717FF0028FAD12046FEF77CFF20467E
:10183000FEF7FEFE002800E009E0F8D10AB02846D5
:1018400070BD4020B2E70220B0E78020AEE7062658
:10185000BAE70126B8E70726B6E70000E01A000855
:10186000000801400024014030B587B00C460160FB
:10187000054601214807FFF759F9FEF767FF124AAD
:1018800004AB07CA07C3BCB15FF01000ADF810008D
:1018900004A90E48FFF766F800200090019002901E
:1018A00003905CB16946FEF75DFF00200121FEF761
:1018B00041FF07B0284630BD2020E7E710206946E9
:1018C000FEF750FF1020F1E7E01A00080008014081
:1018D00010B5044601460248FFF77FFD204610BDC3
:1018E000003801402DE9F04104468CB008306060BA
:1018F00001260025A4F8F85084F8FA6031463046F5
:10190000FFF708F9012144F20400FFF727F9182036
:1019100002904FF49050DFF89880ADF80000022755
:10192000694640460197FFF71DF8482002904FF4A2
:101930004060ADF80000694640460197FFF712F895
:1019400009A8FFF7AEFC1B4F09A93846FFF79AFC20
:1019500003A8FFF737FD4FF4612003904FF4407068
:10196000ADF8180003A93846FFF7D2FC25208DF802
:101970001C008DF81E5004208DF81D0007A8089645
:10198000FFF770F8012240F225513846FFF7A8FC16
:10199000012280213846FFF794FC0748FEF716FF26
:1019A00001213846FFF783FC0CB02046BDE8F081EA
:1019B00000080140003801404400024010B5064CC8
:1019C00002212046FEF73EFE0028F9D02046BDE861
:1019D0001040FEF734BE000000240140B1F5805FE6
:1019E00001D340F6FF71006800284FF0000001D0DD
:1019F000FEF7CCBEFEF7D4BE10B500F001F810BD66
:101A000010B5FEF723FC10BD10B500F001F810BDB5
:101A100010B5040007D1012405E0FEF749FC006879
:101A200000B9044880472046FEF78DFC0028F4D01A
:101A300010BD0000E1030008FEE700F015B800B596
:101A4000CDB06846FFF74EFD00216846FFF7D2FD96
:101A50006846FFF76FFD6846FFF727FD6846FFF70A
:101A600059FD4DB0002000BDC0B20021FFF730BFCE
:101A700010B504468079012802D12068FFF7BCFF29
:101A8000204610BDBFFF3A00A300BEFF4CFED8FFAA
:101A90007103AB01CFFA7DFBE505180840FBDDF4CF
:101AA000D301550CD301DDF440FB1808E5057DFB9F
:101AB000CFFAAB017103D8FF4CFEBEFFA3003A0082
:101AC000BFFF00000000000001000100060000024E
:101AD00000010000040000001000000010000000E1
:101AE00000000000020000001000000000000000E4
:101AF00003000000000000000000000000000000E3
:101B000000000000000006000000000001000000CE
:101B10000000E02E7017B80BE80300000000000082
:101B20000000000015150008000000000000000083
:101B30000000000000000000000000005C1B000826
:101B4000000000205800000028010008B41B000815
:101B50005800002070060000440100080008014001
:101B600000100140001001400000000000000000D3
:101B700004380140000000001000000000000000D8
:101B800000000000800000000000000000000000D5
:101B9000000000000020000000000000000002041F
:101BA0000608000000000102030401020304060706
:041BB0000809000020
:04000005080000ED02
:00000001FF
